:100000006DC0DFC186C085C084C083C082C081C08E
:1000100080C07FC07EC07DC07CC07BC07AC079C0FC
:1000200078C077C076C00403090418037200610029
:10003000700068006E00650074002E006E006500A0
:10004000740018035300650067006100200053002E
:1000500061007400750072006E000A033100300008
:100060003000300005010905A10185010901A10049
:100070000930093109360937150026FF0075089542
:10008000048102C005091901291015002501750117
:1000900095108102C005010902A10185020901A193
:1000A0000005091901290415002501950475018130
:1000B00002950175048103C00501093009311581DC
:1000C000257F750895028106C0120101010000001C
:1000D0000881177E050001010203010011241FBEE3
:1000E000CFE5D4E0DEBFCDBF10E0A0E6B0E0EEE5A6
:1000F000FFE002C005900D92AC39B107D9F711E0CD
:10010000ACE9B0E001C01D92A031B107E1F71AD30C
:1001100024C776CF85B7836085BF8BB780648BBFDC
:1001200083EC8093E60008950F931F93CF93DF93A2
:100130009091F60019160CF0A8C02091F300809160
:10014000F2008D3209F097C08AE5809361009B3000
:1001500009F091C0CCE0D0E0C21BD109C650DF4FFE
:100160008881807609F079C01092E4008981882323
:1001700059F41092E50084EE90E09093F50080939E
:10018000F40030E822E070C0853021F48A81809349
:10019000F70061C0863009F043C08B818130D9F10E
:1001A000823019F4CE0170D25AC0833039F58A8179
:1001B000882349F486E290E09093F5008093F40060
:1001C00030EC24E051C0813019F48AE290E004C0A0
:1001D000823049F482E490E09093F5008093F4003B
:1001E00030EC28E141C08330E9F58AE590E0909356
:1001F000F5008093F40030EC2CE036C0813249F4F5
:100200008FEA90E09093F5008093F40030EC29E0C1
:100210002BC0823239F5CE0137D2282F30EC24C0E2
:10022000883019F489EF90E00AC0893021F48A817E
:100230008093F90010C08A3049F484EE90E09093E6
:10024000F5008093F40030E821E00EC08B3019F403
:1002500083EC8093E60030E806C0CE0143D2282F1D
:1002600030E802C030EC20E08F81882339F48E81A1
:10027000821728F003C030E880E001C0822F30935D
:100280009C00809360001092F6008091610084FFD2
:1002900049C0809160008F3F09F444C0182F893015
:1002A00008F018E0811B8093600080919C0080FD25
:1002B00002C00BE401C003EC8F5F80939C0020918F
:1002C000F4003091F50086FD05C0D901912FECEDC9
:1002D000F0E011C0ACEDB0E080E090E006C0F901C4
:1002E000E80FF91FE491ED9301961817C1F705C0C7
:1002F0008D91819391509923D9F7F901E10FF11D67
:10030000F093F500E093F4008CED90E0612F55D070
:10031000183019F08FEF809360000093DB001C5FB2
:10032000109361009AE080B3857031F49150D9F751
:100330001092F7001092F100DF91CF911F910F9171
:1003400008951F93DC01162F8091620084FF0AC07C
:100350008091E60098E889278093E600912FE7EEE8
:10036000F0E007C08AE580936200F8CF8D91819319
:1003700091509923D9F787EE90E0612F1ED01C5F32
:10038000109362001F910895A82FB92F8FEF9FEF50
:1003900041E050EA615070F02D9138E0722F7827DB
:1003A00096958795269570FF02C0842795273A95E4
:1003B000A9F7F0CF809590950895E6DF8D939D93F2
:1003C0000895CF93CFB7CF93809BFECF809B09C07A
:1003D000809B07C0809B05C0809B03C0809B01C0A1
:1003E0009EC0DF93C091F300DD27C650DF4F809B96
:1003F00002C0DF91EBCF2F930F931F9300B32FEF2A
:1004000000FB20F94F933F9310B34FEF012700FB00
:1004100021F93BE031C04E7F012F10B3216028C08D
:10042000102F4D7F2260000000B329C04B7F246055
:10043000012F000010B32BC010B3477F28602AC0E3
:100440004F7E00B320612CC04F7D10B320622FC0BF
:100450004F7B00B3206432C0422700B349934FEF73
:100460000000102710FB20F910B31570A9F1297FA7
:1004700091F2012700FB21F900B3237F89F231506B
:10048000F0F1102710FB22F910B3277E79F2012733
:1004900000FB23F92F7C81F200B3102710FB24F915
:1004A0002F7971F200C010B3012700FB25F92F73DB
:1004B00059F200C000B3102710FB26F9223040F299
:1004C00000C010B3012700FB27F9243028F64F772E
:1004D000206810B30000F9CF3B503195333010E461
:1004E0001ABFB8F0C31BD0400881033C41F10B3464
:1004F00031F11981412F1F772091F100121731F44A
:10050000093691F10D3279F0013E69F022272093EE
:10051000F8003F914F911F910F912F91DF91CF9153
:10052000CFBFCF9118950093F8003F914F911F9145
:100530000F912F91DF91CAB7C6FD46CFF0CF009142
:10054000F800002331F31091F6001123A1F53430A7
:10055000A2F13093F6000093F2001091F3003BE01B
:10056000311B3093F30029C00091F60001301CF5D7
:100570000AE547FD09C03091610034FD20C00093B9
:100580006100CBEDD0E01FC03091620034FD17C098
:1005900000936200C6EED0E016C0052710E002BB53
:1005A0001FC0052722C0052727C005272CC0052707
:1005B00010E002BB33C04AE503C042ED01C0432F47
:1005C000C4E1D0E032E011B31560909A02B311BBE0
:1005D0005F9355E020E820FF052702BB279517957C
:1005E0001C3FD8F620FF0527279502BB17951C3F17
:1005F000C0F620FF05272795179502BB1C3F98F6EC
:1006000020FF0527279517951C3F02BB70F600C0F9
:10061000499120FF052702BB279517951C3F38F607
:1006200020FF0527279502BB17951C3F38F520FFB3
:1006300005272795179502BB1C3F10F520FF0527BE
:10064000279517951C3F02BBE8F4242F3A9519F61D
:100650000A7F5F9102BB00C01091F700C651D040E5
:1006600011F01093F10010E41ABF016011B31A7F6A
:10067000402F4A7F02BB11BB42BB4BCF0527D3CFD4
:100680000527D8CF0527DDCFFC018081807641F595
:100690008181863029F583818230D1F0823269F000
:1006A0008130F1F48091A1009091A2009093F50027
:1006B0008093F4008091A300089580919E00909112
:1006C0009F009093F5008093F4008091A00008951E
:1006D00083E690E09093F5008093F40082E2089521
:1006E00080E00895DC0126EA30E03093F5002093A5
:1006F000F4008C918076803219F511968C911197C7
:10070000813061F4E091A400F091A5000088F189A6
:10071000E02DC90112966C9109950895823041F43B
:1007200086EB90E09093F5008093F40081E00895CB
:100730008A3031F413968C918093B60080E008954E
:1007400080E008958F929F92AF92BF92CF92DF92F6
:10075000EF92FF920F931F93CF93DF9386B333D122
:10076000FC019093A5008093A400848195819093CF
:100770009F0080939E0082818093A0008085918558
:10078000009731F09093A2008093A100868107C06A
:1007900089EC90E09093A2008093A100C5D3809350
:1007A000A3008091A00080937C0014BA8FEF85BBDA
:1007B00088EF82BB85E081BB11BA83BF8FE085BD26
:1007C00084EC83BDE091A400F091A5000284F38540
:1007D000E02D099585B78F7885BF9CDC789400E083
:1007E000FF24F39410E08824839431E0C32ED12CAD
:1007F00020E8922E9CE2A92E91E0B92E02C0FF249F
:100800001E2DA89591DCFF2041F0E091A400F0910D
:10081000A5000484F585E02D099508B600FE0DC0FD
:1008200088BEE090B600EE2041F0153010F403E0F1
:1008300005C08BEFE82EE10E01C0E12E08B607FEE1
:1008400033C098BE002399F585B7806885BF889529
:1008500085B78F7785BFC5010197F1F7E091A400B7
:10086000F091A5000484F585E02D0995C0E0D0E065
:1008700012C00684F785E02D9E012F5F822F099517
:10088000882341F0C6010C2E02C0880F991F0A94DC
:10089000E2F7082B2196E091A400F091A500808159
:1008A0009181C817D9072CF3002309F4A8CFC0E021
:1008B000D0E02DC0802F992787FD90950C2E02C087
:1008C000959587950A94E2F780FF20C0CE018F5F4F
:1008D000682F0088F189E02D86EA90E00995182FAD
:1008E00001C022DC8091620084FFFBCF612F77275B
:1008F00067FD709586EA90E024DDC6010C2E02C0EB
:10090000880F991F0A94E2F7809508232196E091B9
:10091000A400F091A50080819181C817D90754F2F5
:100920006ECF43B366B350E0CA0184709070959562
:1009300087959A0128703070E3E035952795EA9500
:10094000E1F7822B9A0122703070220F331F822B25
:100950004170507023E0440F551F2A95E1F7842B16
:1009600070E06072707075956795862B08958FB7EB
:10097000F89490E394BB9FEF95BB17BA98BB8FBFD9
:1009800008950F931F93882319F414E604E011C00F
:1009900014E604E005C0802F8A95F1F7115069F044
:1009A000C0DF84FFF8CF0BC0802F8A95F1F711507C
:1009B00021F0B7DF84FDF8CF02C08FEF01C080E0E7
:1009C0001F910F91089584E690E090938A008093A0
:1009D000890085E890E008951F93162F115012307A
:1009E00010F010E029C0009789F0E12FF0E0E956FF
:1009F000FF4FE081FF27E7FDF09529E0129F90016E
:100A0000112429543F4FB901AF019ED229E0129F12
:100A100090011124E12FF0E0E956FF4F1081A90168
:100A200047535F4FE12FFF27E7FDF09529543F4FD4
:100A3000CA01B901AF0188D2812F1F910895E82F13
:100A40008091990090919A00892B31F010929A0030
:100A50001092990081E008958E2F8150823010F01D
:100A600080E0089569E0869FB0011124E82FF0E04E
:100A7000E956FF4F4081552747FD5095CB018954DA
:100A80009F4F67537F4F53D208959F92AF92BF926B
:100A9000CF92DF92EF92FF920F931F93DF93CF934A
:100AA000CDB7DEB7A0970FB6F894DEBF0FBECDBFAF
:100AB000AD9AAC9A30E1F32E8F2D8A95F1F731DFA4
:100AC000982F813109F0F2C089E0E0ECF0E0DF011D
:100AD0001D928A95E9F782E08093C0008F2D8A9558
:100AE000F1F7AD988F2D8A95F1F7FF2400E010E023
:100AF0002EE0C22ED12CEE2498E0992E5E010894AF
:100B0000A11CB11CFF2019F0AC9A81E002C0AC9886
:100B100080E037DF882309F0F5C1892D8A95F1F748
:100B200000DFF501E00FF11F80830115110541F091
:100B30008A81823129F488E0C82ED12CEE24E394F6
:100B40000F5F1F4F0C151D051CF481E0F826DACF4E
:100B500091E09093B7008FE78093B8008093B9003D
:100B60008093BA008093BB001092BC001092BD002D
:100B70008C81282F82FD02C09093BC0020FD05C00F
:100B80008091BC0082608093BC0021FD05C08091F3
:100B9000BC0084608093BC008D81982F82FD05C0CD
:100BA0008091BC0088608093BC0091FD05C080915D
:100BB000BC0080618093BC0090FD05C08091BC00AA
:100BC00080628093BC0023FD05C08091BC008064DE
:100BD0008093BC008E8183FD05C08091BC0080683D
:100BE0008093BC0093FD05C08091BD00816080931F
:100BF000BD008B81EE20A1F0982F83FD03C08FEF05
:100C00008093B80092FD02C01092B80091FD03C01D
:100C10008FEF8093B90090FD40C01092B9003DC0A5
:100C2000982F83FD05C08091BD0082608093BD0038
:100C300092FD05C08091BD0084608093BD0091FD50
:100C400005C08091BD0088608093BD0090FD05C007
:100C50008091BD0080618093BD009F819295907FBF
:100C600088858F70982B9093B80099859295907F86
:100C70008A858F70982B9093B9009B859295907F71
:100C80008C858F70982B9093BA009D859295907F5C
:100C90008E858F70982B9093BB00AC9A80E1982F33
:100CA0009A95F1F7AD9A8A95F1F72CC18771843145
:100CB00009F08EC000EC10E089E0F80111928A95ED
:100CC000E9F782E08093C00009501040AD9AAC9AD9
:100CD0008F2D8A95F1F725DEE82EAD98AC988F2DF3
:100CE0008A95F1F71EDEC82EAD9AAC988F2D8A95A5
:100CF000F1F717DED82EAD98AC9A8F2D8A95F1F7C3
:100D000010DE91E09093B7009FE79093B800909326
:100D1000B900D80113969C93139714969C93109244
:100D2000BC001092BD00282F83FD03C08FEF80937D
:100D3000B80022FD02C01092B80021FD03C08FEF61
:100D40008093B90020FD02C01092B9002D2DD2FC75
:100D500005C08091BC0081608093BC0020FD05C06F
:100D60008091BC0082608093BC0021FD05C0809111
:100D7000BC0084608093BC009C2DC2FC05C08091A7
:100D8000BC0088608093BC0091FD05C08091BC00D0
:100D900080618093BC0090FD05C08091BC008062A2
:100DA0008093BC0023FD05C08091BC0080648093CB
:100DB000BC00E3FC05C08091BC0080688093BC004F
:100DC00093FDA0C08091BD0081608093BD009AC05A
:100DD000E7EBF0E0903109F07CC081E08093B70050
:100DE0008FE78093B8008093B9008093BA00809316
:100DF000BB001092BC001092BD00892F8A95F1F7BC
:100E0000AD98892F8A95F1F78E010F5F1F4FFF2450
:100E1000B8E0BB2EA9E0CA2ED12CCC0EDD1EFF20DF
:100E200019F0AC9A81E002C0AC9880E0AADD88237A
:100E300009F068C08B2D8A95F1F773DDF801819375
:100E40008F01EC15FD0519F081E0F826E8CFAC9A8A
:100E500080E1982F9A95F1F7AD9A8A95F1F789E09C
:100E6000E0ECF0E0DF011D928A95E9F782E08093E3
:100E7000C0008C81982F80FF05C08091C1008160E7
:100E80008093C10091FF05C08091C1008260809372
:100E9000C10092FF05C08091C10084608093C100B1
:100EA00093FF05C08091C10088608093C1002F81AD
:100EB0002295207F88858F70282B9D819295907F29
:100EC0008E818F70982B9093C20021952093C30040
:100ED00019C081E08093B7008FE78093B8008093BA
:100EE000B9008093BA008093BB001092BC001092AE
:100EF000BD00399689E0DF011D928A95E9F782E00D
:100F00008093C000A0960FB6F894DEBF0FBECDBF91
:100F1000CF91DF911F910F91FF90EF90DF90CF90D5
:100F2000BF90AF909F90089582E190E00895FB01FB
:100F3000DC0104C08D910190801921F44150504092
:100F4000C8F7881B990B0895FB01DC0102C00190D2
:0E0F50000D9241505040D8F70895F894FFCF0D
:100F5E00FF5A5A09022200010100803209040000E2
:100F6E000103000000092101010001220000070514
:100F7E00810308000A02006500000000000000B7AF
:0C0F8E000445051F05EC040704010000E9
:00000001FF
